 attach

 Timestamp is 14f928b2 (reproducible build file hash)

 Preferred load address is 0000000180000000

 Start         Length     Name                   Class
 0001:00000000 00001c70H .text$mn                CODE
 0001:00001c70 00000036H .text$mn$00             CODE
 0001:00001ca6 00000092H .text$x                 CODE
 0002:00000000 00000270H .idata$5                DATA
 0002:00000270 00000038H .00cfg                  DATA
 0002:000002a8 00000008H .CRT$XCA                DATA
 0002:000002b0 00000008H .CRT$XCZ                DATA
 0002:000002b8 00000008H .CRT$XIA                DATA
 0002:000002c0 00000008H .CRT$XIZ                DATA
 0002:000002c8 00000008H .CRT$XPA                DATA
 0002:000002d0 00000008H .CRT$XPZ                DATA
 0002:000002d8 00000008H .CRT$XTA                DATA
 0002:000002e0 00000010H .CRT$XTZ                DATA
 0002:000002e8 00000000H .gehcont$y              DATA
 0002:000002e8 00000000H .gfids$y                DATA
 0002:000002f0 00000510H .rdata                  DATA
 0002:00000800 00000000H .rdata$CastGuardVftablesA DATA
 0002:00000800 00000000H .rdata$CastGuardVftablesC DATA
 0002:00000800 0000006cH .rdata$voltmd           DATA
 0002:0000086c 000002b4H .rdata$zzzdbg           DATA
 0002:00000b20 00000008H .rtc$IAA                DATA
 0002:00000b28 00000008H .rtc$IZZ                DATA
 0002:00000b30 00000008H .rtc$TAA                DATA
 0002:00000b38 00000008H .rtc$TZZ                DATA
 0002:00000b40 000002d0H .xdata                  DATA
 0002:00000e10 00000364H .edata                  DATA
 0002:00001174 000000b4H .idata$2                DATA
 0002:00001228 00000018H .idata$3                DATA
 0002:00001240 00000270H .idata$4                DATA
 0002:000014b0 0000066aH .idata$6                DATA
 0003:00000000 00000040H .data                   DATA
 0003:00000040 00000608H .bss                    DATA
 0004:00000000 00000270H .pdata                  DATA
 0005:00000000 00000060H .rsrc$01                DATA
 0005:00000060 00000310H .rsrc$02                DATA

  Address         Publics by Value              Rva+Base               Lib:Object

 0000:00000000       __AbsoluteZero             0000000000000000     <absolute>
 0000:00000000       ___safe_se_handler_count   0000000000000000     <absolute>
 0000:00000000       ___safe_se_handler_table   0000000000000000     <absolute>
 0000:00000000       __arm64x_extra_rfe_table   0000000000000000     <absolute>
 0000:00000000       __arm64x_extra_rfe_table_size 0000000000000000     <absolute>
 0000:00000000       __arm64x_native_entrypoint 0000000000000000     <absolute>
 0000:00000000       __arm64x_redirection_metadata 0000000000000000     <absolute>
 0000:00000000       __arm64x_redirection_metadata_count 0000000000000000     <absolute>
 0000:00000000       __dynamic_value_reloc_table 0000000000000000     <absolute>
 0000:00000000       __enclave_config           0000000000000000     <absolute>
 0000:00000000       __guard_check_icall_a64n_fptr 0000000000000000     <absolute>
 0000:00000000       __guard_eh_cont_count      0000000000000000     <absolute>
 0000:00000000       __guard_eh_cont_table      0000000000000000     <absolute>
 0000:00000000       __guard_fids_count         0000000000000000     <absolute>
 0000:00000000       __guard_fids_table         0000000000000000     <absolute>
 0000:00000000       __guard_iat_count          0000000000000000     <absolute>
 0000:00000000       __guard_iat_table          0000000000000000     <absolute>
 0000:00000000       __guard_longjmp_count      0000000000000000     <absolute>
 0000:00000000       __guard_longjmp_table      0000000000000000     <absolute>
 0000:00000000       __hybrid_auxiliary_delayload_iat 0000000000000000     <absolute>
 0000:00000000       __hybrid_auxiliary_delayload_iat_copy 0000000000000000     <absolute>
 0000:00000000       __hybrid_auxiliary_iat     0000000000000000     <absolute>
 0000:00000000       __hybrid_auxiliary_iat_copy 0000000000000000     <absolute>
 0000:00000000       __hybrid_code_map          0000000000000000     <absolute>
 0000:00000000       __hybrid_code_map_count    0000000000000000     <absolute>
 0000:00000000       __hybrid_image_info_bitfield 0000000000000000     <absolute>
 0000:00000000       __x64_code_ranges_to_entry_points 0000000000000000     <absolute>
 0000:00000000       __x64_code_ranges_to_entry_points_count 0000000000000000     <absolute>
 0000:00000100       __guard_flags              0000000000000100     <absolute>
 0000:00000000       __ImageBase                0000000180000000     <linker-defined>
 0001:00000000       Java_sun_tools_attach_AttachProviderImpl_enumProcesses 0000000180001000 f   AttachProviderImpl.obj
 0001:00000088       Java_sun_tools_attach_AttachProviderImpl_isLibraryLoadedByProcess 0000000180001088 f   AttachProviderImpl.obj
 0001:000001cc       Java_sun_tools_attach_AttachProviderImpl_tempPath 00000001800011cc f   AttachProviderImpl.obj
 0001:00000288       Java_sun_tools_attach_AttachProviderImpl_volumeFlags 0000000180001288 f   AttachProviderImpl.obj
 0001:0000031c       Java_sun_tools_attach_VirtualMachineImpl_closePipe 000000018000131c f   VirtualMachineImpl.obj
 0001:0000031c       Java_sun_tools_attach_VirtualMachineImpl_closeProcess 000000018000131c f   VirtualMachineImpl.obj
 0001:00000328       Java_sun_tools_attach_VirtualMachineImpl_connectPipe 0000000180001328 f   VirtualMachineImpl.obj
 0001:00000364       Java_sun_tools_attach_VirtualMachineImpl_createPipe 0000000180001364 f   VirtualMachineImpl.obj
 0001:0000045c       Java_sun_tools_attach_VirtualMachineImpl_enqueue 000000018000145c f   VirtualMachineImpl.obj
 0001:00000880       Java_sun_tools_attach_VirtualMachineImpl_generateStub 0000000180001880 f   VirtualMachineImpl.obj
 0001:000008f0       Java_sun_tools_attach_VirtualMachineImpl_init 00000001800018f0 f   VirtualMachineImpl.obj
 0001:0000091c       Java_sun_tools_attach_VirtualMachineImpl_openProcess 000000018000191c f   VirtualMachineImpl.obj
 0001:00000aa8       Java_sun_tools_attach_VirtualMachineImpl_readPipe 0000000180001aa8 f   VirtualMachineImpl.obj
 0001:00000b7c       __local_stdio_printf_options 0000000180001b7c f i VirtualMachineImpl.obj
 0001:00000d8c       jvm_attach_thread_func     0000000180001d8c f   VirtualMachineImpl.obj
 0001:00000e14       _guard_check_icall_nop     0000000180001e14 f   MSVCRT:guard_support.obj
 0001:00000e14       jvm_attach_thread_func_end 0000000180001e14 f   VirtualMachineImpl.obj
 0001:00000e18       sprintf                    0000000180001e18 f i VirtualMachineImpl.obj
 0001:00000e6f       JNU_NewStringPlatform      0000000180001e6f f   java:java.dll
 0001:00000e75       JNU_GetStringPlatformChars 0000000180001e75 f   java:java.dll
 0001:00000e7b       JNU_ReleaseStringPlatformChars 0000000180001e7b f   java:java.dll
 0001:00000e81       JNU_ThrowByName            0000000180001e81 f   java:java.dll
 0001:00000e87       JNU_ThrowInternalError     0000000180001e87 f   java:java.dll
 0001:00000e8d       JNU_ThrowIOException       0000000180001e8d f   java:java.dll
 0001:00000e93       JNU_ThrowIOExceptionWithLastError 0000000180001e93 f   java:java.dll
 0001:00000e99       ConvertStringSecurityDescriptorToSecurityDescriptorA 0000000180001e99 f   advapi32:ADVAPI32.dll
 0001:00000e9f       EnumProcesses              0000000180001e9f f   psapi:PSAPI.DLL
 0001:00000ea5       EnumProcessModules         0000000180001ea5 f   psapi:PSAPI.DLL
 0001:00000eab       GetModuleBaseNameA         0000000180001eab f   psapi:PSAPI.DLL
 0001:00000eb4       __GSHandlerCheck           0000000180001eb4 f   MSVCRT:gshandler.obj
 0001:00000ed4       __GSHandlerCheckCommon     0000000180001ed4 f   MSVCRT:gshandler.obj
 0001:00000f40       __security_check_cookie    0000000180001f40 f   MSVCRT:amdsecgs.obj
 0001:00001280       _DllMainCRTStartup         0000000180002280 f   MSVCRT:dll_dllmain.obj
 0001:000012c0       __raise_securityfailure    00000001800022c0 f   MSVCRT:gs_report.obj
 0001:000012f4       __report_gsfailure         00000001800022f4 f   MSVCRT:gs_report.obj
 0001:0000143c       __security_init_cookie     000000018000243c f   MSVCRT:gs_support.obj
 0001:000014e8       DllMain                    00000001800024e8 f   MSVCRT:dll_dllmain_stub.obj
 0001:0000150c       ?__scrt_initialize_type_info@@YAXXZ 000000018000250c f   MSVCRT:tncleanup.obj
 0001:0000151c       ?__scrt_uninitialize_type_info@@YAXXZ 000000018000251c f   MSVCRT:tncleanup.obj
 0001:00001528       __local_stdio_scanf_options 0000000180002528 f i MSVCRT:default_local_stdio_options.obj
 0001:00001530       __scrt_initialize_default_local_stdio_options 0000000180002530 f   MSVCRT:default_local_stdio_options.obj
 0001:0000154c       __scrt_acquire_startup_lock 000000018000254c f   MSVCRT:utility.obj
 0001:00001588       __scrt_dllmain_after_initialize_c 0000000180002588 f   MSVCRT:utility.obj
 0001:000015bc       __scrt_dllmain_before_initialize_c 00000001800025bc f   MSVCRT:utility.obj
 0001:000015d4       __scrt_dllmain_crt_thread_attach 00000001800025d4 f   MSVCRT:utility.obj
 0001:000015fc       __scrt_dllmain_crt_thread_detach 00000001800025fc f   MSVCRT:utility.obj
 0001:00001614       __scrt_dllmain_exception_filter 0000000180002614 f   MSVCRT:utility.obj
 0001:00001674       __scrt_dllmain_uninitialize_c 0000000180002674 f   MSVCRT:utility.obj
 0001:000016a4       __scrt_dllmain_uninitialize_critical 00000001800026a4 f   MSVCRT:utility.obj
 0001:000016b8       __scrt_initialize_crt      00000001800026b8 f   MSVCRT:utility.obj
 0001:00001704       __scrt_initialize_onexit_tables 0000000180002704 f   MSVCRT:utility.obj
 0001:00001790       __scrt_is_nonwritable_in_current_image 0000000180002790 f   MSVCRT:utility.obj
 0001:00001828       __scrt_release_startup_lock 0000000180002828 f   MSVCRT:utility.obj
 0001:0000184c       __scrt_uninitialize_crt    000000018000284c f   MSVCRT:utility.obj
 0001:00001878       __scrt_get_dyn_tls_init_callback 0000000180002878 f   MSVCRT:dyn_tls_init.obj
 0001:00001880       __crt_debugger_hook        0000000180002880 f   MSVCRT:utility_desktop.obj
 0001:00001888       __scrt_fastfail            0000000180002888 f   MSVCRT:utility_desktop.obj
 0001:000019d4       _RTC_Initialize            00000001800029d4 f   MSVCRT:initsect.obj
 0001:00001a10       _RTC_Terminate             0000000180002a10 f   MSVCRT:initsect.obj
 0001:00001a4c       __isa_available_init       0000000180002a4c f   MSVCRT:cpu_disp.obj
 0001:00001bf8       _get_startup_argv_mode     0000000180002bf8 f   MSVCRT:argv_mode.obj
 0001:00001c00       __scrt_is_ucrt_dll_in_use  0000000180002c00 f   MSVCRT:ucrt_detection.obj
 0001:00001c10       memset                     0000000180002c10 f   vcruntime:VCRUNTIME140.dll
 0001:00001c16       __C_specific_handler       0000000180002c16 f   vcruntime:VCRUNTIME140.dll
 0001:00001c1c       __std_type_info_destroy_list 0000000180002c1c f   vcruntime:VCRUNTIME140.dll
 0001:00001c22       strcmp                     0000000180002c22 f   ucrt:api-ms-win-crt-string-l1-1-0.dll
 0001:00001c28       strcpy                     0000000180002c28 f   ucrt:api-ms-win-crt-string-l1-1-0.dll
 0001:00001c2e       _initterm                  0000000180002c2e f   ucrt:api-ms-win-crt-runtime-l1-1-0.dll
 0001:00001c34       _initterm_e                0000000180002c34 f   ucrt:api-ms-win-crt-runtime-l1-1-0.dll
 0001:00001c3a       _seh_filter_dll            0000000180002c3a f   ucrt:api-ms-win-crt-runtime-l1-1-0.dll
 0001:00001c40       _configure_narrow_argv     0000000180002c40 f   ucrt:api-ms-win-crt-runtime-l1-1-0.dll
 0001:00001c46       _initialize_narrow_environment 0000000180002c46 f   ucrt:api-ms-win-crt-runtime-l1-1-0.dll
 0001:00001c4c       _initialize_onexit_table   0000000180002c4c f   ucrt:api-ms-win-crt-runtime-l1-1-0.dll
 0001:00001c52       _execute_onexit_table      0000000180002c52 f   ucrt:api-ms-win-crt-runtime-l1-1-0.dll
 0001:00001c58       _cexit                     0000000180002c58 f   ucrt:api-ms-win-crt-runtime-l1-1-0.dll
 0001:00001c60       __acrt_initialize          0000000180002c60 f   MSVCRT:ucrt_stubs.obj
 0001:00001c60       __acrt_thread_attach       0000000180002c60 f   MSVCRT:ucrt_stubs.obj
 0001:00001c60       __acrt_thread_detach       0000000180002c60 f   MSVCRT:ucrt_stubs.obj
 0001:00001c60       __acrt_uninitialize        0000000180002c60 f   MSVCRT:ucrt_stubs.obj
 0001:00001c60       __acrt_uninitialize_critical 0000000180002c60 f   MSVCRT:ucrt_stubs.obj
 0001:00001c60       __scrt_stub_for_acrt_initialize 0000000180002c60 f   MSVCRT:ucrt_stubs.obj
 0001:00001c60       __scrt_stub_for_acrt_thread_attach 0000000180002c60 f   MSVCRT:ucrt_stubs.obj
 0001:00001c60       __scrt_stub_for_acrt_thread_detach 0000000180002c60 f   MSVCRT:ucrt_stubs.obj
 0001:00001c60       __scrt_stub_for_acrt_uninitialize 0000000180002c60 f   MSVCRT:ucrt_stubs.obj
 0001:00001c60       __scrt_stub_for_acrt_uninitialize_critical 0000000180002c60 f   MSVCRT:ucrt_stubs.obj
 0001:00001c60       __vcrt_initialize          0000000180002c60 f   MSVCRT:ucrt_stubs.obj
 0001:00001c60       __vcrt_thread_attach       0000000180002c60 f   MSVCRT:ucrt_stubs.obj
 0001:00001c60       __vcrt_thread_detach       0000000180002c60 f   MSVCRT:ucrt_stubs.obj
 0001:00001c60       __vcrt_uninitialize        0000000180002c60 f   MSVCRT:ucrt_stubs.obj
 0001:00001c60       __vcrt_uninitialize_critical 0000000180002c60 f   MSVCRT:ucrt_stubs.obj
 0001:00001c64       __scrt_stub_for_is_c_termination_complete 0000000180002c64 f   MSVCRT:ucrt_stubs.obj
 0001:00001c64       _is_c_termination_complete 0000000180002c64 f   MSVCRT:ucrt_stubs.obj
 0001:00001c67       memcpy                     0000000180002c67 f   vcruntime:VCRUNTIME140.dll
 0001:00001c80       _guard_dispatch_icall_nop  0000000180002c80 f   MSVCRT:guard_dispatch.obj
 0001:00001ca0       _guard_xfg_dispatch_icall_nop 0000000180002ca0 f   MSVCRT:guard_xfg_dispatch.obj
 0002:00000000       __imp_LookupPrivilegeValueA 0000000180003000     advapi32:ADVAPI32.dll
 0002:00000008       __imp_ImpersonateSelf      0000000180003008     advapi32:ADVAPI32.dll
 0002:00000010       __imp_AdjustTokenPrivileges 0000000180003010     advapi32:ADVAPI32.dll
 0002:00000018       __imp_OpenThreadToken      0000000180003018     advapi32:ADVAPI32.dll
 0002:00000020       __imp_ConvertStringSecurityDescriptorToSecurityDescriptorA 0000000180003020     advapi32:ADVAPI32.dll
 0002:00000028       \177ADVAPI32_NULL_THUNK_DATA 0000000180003028     advapi32:ADVAPI32.dll
 0002:00000030       __imp_GetSystemTimeAsFileTime 0000000180003030     kernel32:KERNEL32.dll
 0002:00000038       __imp_DisableThreadLibraryCalls 0000000180003038     kernel32:KERNEL32.dll
 0002:00000040       __imp_InitializeSListHead  0000000180003040     kernel32:KERNEL32.dll
 0002:00000048       __imp_IsDebuggerPresent    0000000180003048     kernel32:KERNEL32.dll
 0002:00000050       __imp_QueryPerformanceCounter 0000000180003050     kernel32:KERNEL32.dll
 0002:00000058       __imp_GetCurrentThreadId   0000000180003058     kernel32:KERNEL32.dll
 0002:00000060       __imp_RtlVirtualUnwind     0000000180003060     kernel32:KERNEL32.dll
 0002:00000068       __imp_IsProcessorFeaturePresent 0000000180003068     kernel32:KERNEL32.dll
 0002:00000070       __imp_TerminateProcess     0000000180003070     kernel32:KERNEL32.dll
 0002:00000078       __imp_SetUnhandledExceptionFilter 0000000180003078     kernel32:KERNEL32.dll
 0002:00000080       __imp_UnhandledExceptionFilter 0000000180003080     kernel32:KERNEL32.dll
 0002:00000088       __imp_GetTempPathA         0000000180003088     kernel32:KERNEL32.dll
 0002:00000090       __imp_GetVolumeInformationA 0000000180003090     kernel32:KERNEL32.dll
 0002:00000098       __imp_CloseHandle          0000000180003098     kernel32:KERNEL32.dll
 0002:000000a0       __imp_OpenProcess          00000001800030a0     kernel32:KERNEL32.dll
 0002:000000a8       __imp_ReadFile             00000001800030a8     kernel32:KERNEL32.dll
 0002:000000b0       __imp_DuplicateHandle      00000001800030b0     kernel32:KERNEL32.dll
 0002:000000b8       __imp_GetLastError         00000001800030b8     kernel32:KERNEL32.dll
 0002:000000c0       __imp_SetLastError         00000001800030c0     kernel32:KERNEL32.dll
 0002:000000c8       __imp_ConnectNamedPipe     00000001800030c8     kernel32:KERNEL32.dll
 0002:000000d0       __imp_WaitForSingleObject  00000001800030d0     kernel32:KERNEL32.dll
 0002:000000d8       __imp_GetCurrentProcess    00000001800030d8     kernel32:KERNEL32.dll
 0002:000000e0       __imp_GetCurrentProcessId  00000001800030e0     kernel32:KERNEL32.dll
 0002:000000e8       __imp_CreateRemoteThread   00000001800030e8     kernel32:KERNEL32.dll
 0002:000000f0       __imp_GetCurrentThread     00000001800030f0     kernel32:KERNEL32.dll
 0002:000000f8       __imp_GetExitCodeThread    00000001800030f8     kernel32:KERNEL32.dll
 0002:00000100       __imp_VirtualAllocEx       0000000180003100     kernel32:KERNEL32.dll
 0002:00000108       __imp_WriteProcessMemory   0000000180003108     kernel32:KERNEL32.dll
 0002:00000110       __imp_VirtualFreeEx        0000000180003110     kernel32:KERNEL32.dll
 0002:00000118       __imp_IsWow64Process       0000000180003118     kernel32:KERNEL32.dll
 0002:00000120       __imp_GetModuleHandleA     0000000180003120     kernel32:KERNEL32.dll
 0002:00000128       __imp_GetProcAddress       0000000180003128     kernel32:KERNEL32.dll
 0002:00000130       __imp_LocalFree            0000000180003130     kernel32:KERNEL32.dll
 0002:00000138       __imp_CreateNamedPipeA     0000000180003138     kernel32:KERNEL32.dll
 0002:00000140       __imp_RtlCaptureContext    0000000180003140     kernel32:KERNEL32.dll
 0002:00000148       __imp_RtlLookupFunctionEntry 0000000180003148     kernel32:KERNEL32.dll
 0002:00000150       \177KERNEL32_NULL_THUNK_DATA 0000000180003150     kernel32:KERNEL32.dll
 0002:00000158       __imp_EnumProcessModules   0000000180003158     psapi:PSAPI.DLL
 0002:00000160       __imp_EnumProcesses        0000000180003160     psapi:PSAPI.DLL
 0002:00000168       __imp_GetModuleBaseNameA   0000000180003168     psapi:PSAPI.DLL
 0002:00000170       \177PSAPI_NULL_THUNK_DATA  0000000180003170     psapi:PSAPI.DLL
 0002:00000178       __imp_memset               0000000180003178     vcruntime:VCRUNTIME140.dll
 0002:00000180       __imp___C_specific_handler 0000000180003180     vcruntime:VCRUNTIME140.dll
 0002:00000188       __imp___std_type_info_destroy_list 0000000180003188     vcruntime:VCRUNTIME140.dll
 0002:00000190       __imp_memcpy               0000000180003190     vcruntime:VCRUNTIME140.dll
 0002:00000198       \177VCRUNTIME140_NULL_THUNK_DATA 0000000180003198     vcruntime:VCRUNTIME140.dll
 0002:000001a0       __imp_malloc               00000001800031a0     ucrt:api-ms-win-crt-heap-l1-1-0.dll
 0002:000001a8       __imp_free                 00000001800031a8     ucrt:api-ms-win-crt-heap-l1-1-0.dll
 0002:000001b0       \177api-ms-win-crt-heap-l1-1-0_NULL_THUNK_DATA 00000001800031b0     ucrt:api-ms-win-crt-heap-l1-1-0.dll
 0002:000001b8       __imp__execute_onexit_table 00000001800031b8     ucrt:api-ms-win-crt-runtime-l1-1-0.dll
 0002:000001c0       __imp__cexit               00000001800031c0     ucrt:api-ms-win-crt-runtime-l1-1-0.dll
 0002:000001c8       __imp__initterm_e          00000001800031c8     ucrt:api-ms-win-crt-runtime-l1-1-0.dll
 0002:000001d0       __imp__initialize_onexit_table 00000001800031d0     ucrt:api-ms-win-crt-runtime-l1-1-0.dll
 0002:000001d8       __imp__initialize_narrow_environment 00000001800031d8     ucrt:api-ms-win-crt-runtime-l1-1-0.dll
 0002:000001e0       __imp__configure_narrow_argv 00000001800031e0     ucrt:api-ms-win-crt-runtime-l1-1-0.dll
 0002:000001e8       __imp__initterm            00000001800031e8     ucrt:api-ms-win-crt-runtime-l1-1-0.dll
 0002:000001f0       __imp__seh_filter_dll      00000001800031f0     ucrt:api-ms-win-crt-runtime-l1-1-0.dll
 0002:000001f8       \177api-ms-win-crt-runtime-l1-1-0_NULL_THUNK_DATA 00000001800031f8     ucrt:api-ms-win-crt-runtime-l1-1-0.dll
 0002:00000200       __imp___stdio_common_vsprintf 0000000180003200     ucrt:api-ms-win-crt-stdio-l1-1-0.dll
 0002:00000208       \177api-ms-win-crt-stdio-l1-1-0_NULL_THUNK_DATA 0000000180003208     ucrt:api-ms-win-crt-stdio-l1-1-0.dll
 0002:00000210       __imp_strcpy               0000000180003210     ucrt:api-ms-win-crt-string-l1-1-0.dll
 0002:00000218       __imp_strcmp               0000000180003218     ucrt:api-ms-win-crt-string-l1-1-0.dll
 0002:00000220       __imp_strncpy              0000000180003220     ucrt:api-ms-win-crt-string-l1-1-0.dll
 0002:00000228       \177api-ms-win-crt-string-l1-1-0_NULL_THUNK_DATA 0000000180003228     ucrt:api-ms-win-crt-string-l1-1-0.dll
 0002:00000230       __imp_JNU_ThrowInternalError 0000000180003230     java:java.dll
 0002:00000238       __imp_JNU_ThrowIOException 0000000180003238     java:java.dll
 0002:00000240       __imp_JNU_GetStringPlatformChars 0000000180003240     java:java.dll
 0002:00000248       __imp_JNU_ThrowIOExceptionWithLastError 0000000180003248     java:java.dll
 0002:00000250       __imp_JNU_ThrowByName      0000000180003250     java:java.dll
 0002:00000258       __imp_JNU_ReleaseStringPlatformChars 0000000180003258     java:java.dll
 0002:00000260       __imp_JNU_NewStringPlatform 0000000180003260     java:java.dll
 0002:00000268       \177java_NULL_THUNK_DATA   0000000180003268     java:java.dll
 0002:00000270       __guard_check_icall_fptr   0000000180003270     MSVCRT:guard_support.obj
 0002:00000278       __guard_xfg_check_icall_fptr 0000000180003278     MSVCRT:guard_support.obj
 0002:00000280       __guard_dispatch_icall_fptr 0000000180003280     MSVCRT:guard_support.obj
 0002:00000288       __guard_xfg_dispatch_icall_fptr 0000000180003288     MSVCRT:guard_support.obj
 0002:00000290       __guard_xfg_table_dispatch_icall_fptr 0000000180003290     MSVCRT:guard_support.obj
 0002:00000298       __castguard_check_failure_os_handled_fptr 0000000180003298     MSVCRT:guard_support.obj
 0002:000002a0       __guard_memcpy_fptr        00000001800032a0     vcruntime:softmemtag.obj
 0002:000002a8       __xc_a                     00000001800032a8     MSVCRT:initializers.obj
 0002:000002b0       __xc_z                     00000001800032b0     MSVCRT:initializers.obj
 0002:000002b8       __xi_a                     00000001800032b8     MSVCRT:initializers.obj
 0002:000002c0       __xi_z                     00000001800032c0     MSVCRT:initializers.obj
 0002:000002c8       __xp_a                     00000001800032c8     MSVCRT:initializers.obj
 0002:000002d0       __xp_z                     00000001800032d0     MSVCRT:initializers.obj
 0002:000002d8       __xt_a                     00000001800032d8     MSVCRT:initializers.obj
 0002:000002e0       __xt_z                     00000001800032e0     MSVCRT:initializers.obj
 0002:000002f0       ??_C@_0BA@ENLPPKBN@no?5such?5process@ 00000001800032f0     VirtualMachineImpl.obj
 0002:00000300       ??_C@_0CL@NFJAPLFK@OpenProcess?$CIpid?$DN?$CFd?$CJ?5failed?$DL?5Las@ 0000000180003300     VirtualMachineImpl.obj
 0002:00000330       ??_C@_0DH@HAHNNIB@Unable?5to?5attach?5to?532?9bit?5proc@ 0000000180003330     VirtualMachineImpl.obj
 0002:00000368       ??_C@_0DB@EJHNPKJJ@com?1sun?1tools?1attach?1AttachNotS@ 0000000180003368     VirtualMachineImpl.obj
 0002:000003a0       ??_C@_0DF@KNAJDOAO@D?3?$CIA?$DLOICI?$DLGRGW?$DL?$DL?$DLWD?$CJ?$CIA?$DLOICI?$DLGA?$DL@ 00000001800033a0     VirtualMachineImpl.obj
 0002:000003d8       ??_C@_0BH@HBAPIBAL@CreateNamedPipe?5failed@ 00000001800033d8     VirtualMachineImpl.obj
 0002:000003f0       ??_C@_0BI@BIDFBHOK@ConnectNamedPipe?5failed@ 00000001800033f0     VirtualMachineImpl.obj
 0002:00000408       ??_C@_08KLCHJOKF@ReadFile@ 0000000180003408     VirtualMachineImpl.obj
 0002:00000414       ??_C@_03KAPDGIM@jvm@       0000000180003414     VirtualMachineImpl.obj
 0002:00000418       ??_C@_0BF@GAHKIOOM@JVM_EnqueueOperation@ 0000000180003418     VirtualMachineImpl.obj
 0002:00000430       ??_C@_0BJ@JNPKEMFE@_JVM_EnqueueOperation?$EA20@ 0000000180003430     VirtualMachineImpl.obj
 0002:00000450       ??_C@_0BD@KIBEHICB@Too?5many?5arguments@ 0000000180003450     VirtualMachineImpl.obj
 0002:00000468       ??_C@_0BG@NFBJGHNB@VirtualAllocEx?5failed@ 0000000180003468     VirtualMachineImpl.obj
 0002:00000480       ??_C@_0BL@GJDMIHJJ@WaitForSingleObject?5failed@ 0000000180003480     VirtualMachineImpl.obj
 0002:000004a0       ??_C@_0CF@HNHEBLGO@jvm?4dll?5not?5loaded?5by?5target?5pr@ 00000001800034a0     VirtualMachineImpl.obj
 0002:000004d0       ??_C@_0EN@MDMJHHAL@Unable?5to?5enqueue?5operation?3?5th@ 00000001800034d0     VirtualMachineImpl.obj
 0002:00000520       ??_C@_0CN@CJKONIL@Remote?5thread?5failed?5for?5unknow@ 0000000180003520     VirtualMachineImpl.obj
 0002:00000550       ??_C@_0DJ@JHMCEEDA@Insufficient?5memory?5or?5insuffic@ 0000000180003550     VirtualMachineImpl.obj
 0002:00000590       ??_C@_0BK@FODHPPG@CreateRemoteThread?5failed@ 0000000180003590     VirtualMachineImpl.obj
 0002:000005b0       ??_C@_0BB@ICFLKOPM@SeDebugPrivilege@ 00000001800035b0     VirtualMachineImpl.obj
 0002:000005c8       _pDefaultRawDllMain        00000001800035c8     MSVCRT:dll_dllmain.obj
 0002:000005c8       _pRawDllMain               00000001800035c8     MSVCRT:dll_dllmain.obj
 0002:000005e0       __xmm@ffffffffffffffffffffffffffffffff 00000001800035e0     MSVCRT:utility.obj
 0002:000005f0       _load_config_used          00000001800035f0     MSVCRT:loadcfg.obj
 0002:00000800       __volatile_metadata        0000000180003800     <linker-defined>
 0002:00000b20       __rtc_iaa                  0000000180003b20     MSVCRT:initsect.obj
 0002:00000b28       __rtc_izz                  0000000180003b28     MSVCRT:initsect.obj
 0002:00000b30       __rtc_taa                  0000000180003b30     MSVCRT:initsect.obj
 0002:00000b38       __rtc_tzz                  0000000180003b38     MSVCRT:initsect.obj
 0002:00001174       __IMPORT_DESCRIPTOR_java   0000000180004174     java:java.dll
 0002:00001188       __IMPORT_DESCRIPTOR_ADVAPI32 0000000180004188     advapi32:ADVAPI32.dll
 0002:0000119c       __IMPORT_DESCRIPTOR_PSAPI  000000018000419c     psapi:PSAPI.DLL
 0002:000011b0       __IMPORT_DESCRIPTOR_KERNEL32 00000001800041b0     kernel32:KERNEL32.dll
 0002:000011c4       __IMPORT_DESCRIPTOR_VCRUNTIME140 00000001800041c4     vcruntime:VCRUNTIME140.dll
 0002:000011d8       __IMPORT_DESCRIPTOR_api-ms-win-crt-string-l1-1-0 00000001800041d8     ucrt:api-ms-win-crt-string-l1-1-0.dll
 0002:000011ec       __IMPORT_DESCRIPTOR_api-ms-win-crt-heap-l1-1-0 00000001800041ec     ucrt:api-ms-win-crt-heap-l1-1-0.dll
 0002:00001200       __IMPORT_DESCRIPTOR_api-ms-win-crt-stdio-l1-1-0 0000000180004200     ucrt:api-ms-win-crt-stdio-l1-1-0.dll
 0002:00001214       __IMPORT_DESCRIPTOR_api-ms-win-crt-runtime-l1-1-0 0000000180004214     ucrt:api-ms-win-crt-runtime-l1-1-0.dll
 0002:00001228       __NULL_IMPORT_DESCRIPTOR   0000000180004228     java:java.dll
 0003:00000000       __security_cookie_complement 0000000180005000     MSVCRT:gs_cookie.obj
 0003:00000008       __security_cookie          0000000180005008     MSVCRT:gs_cookie.obj
 0003:00000010       __scrt_native_dllmain_reason 0000000180005010     MSVCRT:utility.obj
 0003:00000018       __isa_available            0000000180005018     MSVCRT:cpu_disp.obj
 0003:0000001c       __isa_enabled              000000018000501c     MSVCRT:cpu_disp.obj
 0003:00000020       __memset_fast_string_threshold 0000000180005020     MSVCRT:cpu_disp.obj
 0003:00000028       __memset_nt_threshold      0000000180005028     MSVCRT:cpu_disp.obj
 0003:00000030       __scrt_ucrt_dll_is_in_use  0000000180005030     MSVCRT:ucrt_stubs.obj
 0003:000005d0       ?__type_info_root_node@@3U__type_info_node@@A 00000001800055d0     MSVCRT:tncleanup.obj
 0003:000005e0       ?_OptionsStorage@?1??__local_stdio_scanf_options@@9@4_KA 00000001800055e0     MSVCRT:default_local_stdio_options.obj
 0003:000005e8       __scrt_current_native_startup_state 00000001800055e8     MSVCRT:utility.obj
 0003:000005f0       __scrt_native_startup_lock 00000001800055f0     MSVCRT:utility.obj
 0003:00000630       __scrt_debugger_hook_flag  0000000180005630     MSVCRT:utility_desktop.obj
 0003:00000634       __favor                    0000000180005634     MSVCRT:cpu_disp.obj
 0003:00000638       ?_OptionsStorage@?1??__local_stdio_printf_options@@9@9 0000000180005638     <common>
 0003:00000640       __dyn_tls_init_callback    0000000180005640     <common>

 entry point at        0001:00001280

 Static symbols

 0000:ffff7000       .debug$S                   0000000180000000     attach.exp
 0000:ffff7000       .debug$S                   0000000180000000     vcruntime:VCRUNTIME140.dll
 0000:ffff7000       .debug$S                   0000000180000000     vcruntime:VCRUNTIME140.dll
 0000:ffff7000       .debug$S                   0000000180000000     vcruntime:VCRUNTIME140.dll
 0000:ffff7000       .debug$S                   0000000180000000     vcruntime:VCRUNTIME140.dll
 0000:ffff7000       .debug$S                   0000000180000000     vcruntime:VCRUNTIME140.dll
 0000:ffff7000       .debug$S                   0000000180000000     vcruntime:VCRUNTIME140.dll
 0000:ffff7000       .debug$S                   0000000180000000     ucrt:api-ms-win-crt-heap-l1-1-0.dll
 0000:ffff7000       .debug$S                   0000000180000000     ucrt:api-ms-win-crt-heap-l1-1-0.dll
 0000:ffff7000       .debug$S                   0000000180000000     ucrt:api-ms-win-crt-runtime-l1-1-0.dll
 0000:ffff7000       .debug$S                   0000000180000000     ucrt:api-ms-win-crt-runtime-l1-1-0.dll
 0000:ffff7000       .debug$S                   0000000180000000     ucrt:api-ms-win-crt-runtime-l1-1-0.dll
 0000:ffff7000       .debug$S                   0000000180000000     ucrt:api-ms-win-crt-runtime-l1-1-0.dll
 0000:ffff7000       .debug$S                   0000000180000000     ucrt:api-ms-win-crt-runtime-l1-1-0.dll
 0000:ffff7000       .debug$S                   0000000180000000     ucrt:api-ms-win-crt-runtime-l1-1-0.dll
 0000:ffff7000       .debug$S                   0000000180000000     ucrt:api-ms-win-crt-runtime-l1-1-0.dll
 0000:ffff7000       .debug$S                   0000000180000000     ucrt:api-ms-win-crt-runtime-l1-1-0.dll
 0000:ffff7000       .debug$S                   0000000180000000     ucrt:api-ms-win-crt-runtime-l1-1-0.dll
 0000:ffff7000       .debug$S                   0000000180000000     ucrt:api-ms-win-crt-runtime-l1-1-0.dll
 0000:ffff7000       .debug$S                   0000000180000000     ucrt:api-ms-win-crt-runtime-l1-1-0.dll
 0000:ffff7000       .debug$S                   0000000180000000     ucrt:api-ms-win-crt-runtime-l1-1-0.dll
 0000:ffff7000       .debug$S                   0000000180000000     ucrt:api-ms-win-crt-stdio-l1-1-0.dll
 0000:ffff7000       .debug$S                   0000000180000000     ucrt:api-ms-win-crt-string-l1-1-0.dll
 0000:ffff7000       .debug$S                   0000000180000000     ucrt:api-ms-win-crt-string-l1-1-0.dll
 0000:ffff7000       .debug$S                   0000000180000000     ucrt:api-ms-win-crt-string-l1-1-0.dll
 0000:ffff7000       .debug$S                   0000000180000000     advapi32:ADVAPI32.dll
 0000:ffff7000       .debug$S                   0000000180000000     advapi32:ADVAPI32.dll
 0000:ffff7000       .debug$S                   0000000180000000     advapi32:ADVAPI32.dll
 0000:ffff7000       .debug$S                   0000000180000000     advapi32:ADVAPI32.dll
 0000:ffff7000       .debug$S                   0000000180000000     advapi32:ADVAPI32.dll
 0000:ffff7000       .debug$S                   0000000180000000     kernel32:KERNEL32.dll
 0000:ffff7000       .debug$S                   0000000180000000     kernel32:KERNEL32.dll
 0000:ffff7000       .debug$S                   0000000180000000     kernel32:KERNEL32.dll
 0000:ffff7000       .debug$S                   0000000180000000     kernel32:KERNEL32.dll
 0000:ffff7000       .debug$S                   0000000180000000     kernel32:KERNEL32.dll
 0000:ffff7000       .debug$S                   0000000180000000     kernel32:KERNEL32.dll
 0000:ffff7000       .debug$S                   0000000180000000     kernel32:KERNEL32.dll
 0000:ffff7000       .debug$S                   0000000180000000     kernel32:KERNEL32.dll
 0000:ffff7000       .debug$S                   0000000180000000     kernel32:KERNEL32.dll
 0000:ffff7000       .debug$S                   0000000180000000     kernel32:KERNEL32.dll
 0000:ffff7000       .debug$S                   0000000180000000     kernel32:KERNEL32.dll
 0000:ffff7000       .debug$S                   0000000180000000     kernel32:KERNEL32.dll
 0000:ffff7000       .debug$S                   0000000180000000     kernel32:KERNEL32.dll
 0000:ffff7000       .debug$S                   0000000180000000     kernel32:KERNEL32.dll
 0000:ffff7000       .debug$S                   0000000180000000     kernel32:KERNEL32.dll
 0000:ffff7000       .debug$S                   0000000180000000     kernel32:KERNEL32.dll
 0000:ffff7000       .debug$S                   0000000180000000     kernel32:KERNEL32.dll
 0000:ffff7000       .debug$S                   0000000180000000     kernel32:KERNEL32.dll
 0000:ffff7000       .debug$S                   0000000180000000     kernel32:KERNEL32.dll
 0000:ffff7000       .debug$S                   0000000180000000     kernel32:KERNEL32.dll
 0000:ffff7000       .debug$S                   0000000180000000     kernel32:KERNEL32.dll
 0000:ffff7000       .debug$S                   0000000180000000     kernel32:KERNEL32.dll
 0000:ffff7000       .debug$S                   0000000180000000     kernel32:KERNEL32.dll
 0000:ffff7000       .debug$S                   0000000180000000     kernel32:KERNEL32.dll
 0000:ffff7000       .debug$S                   0000000180000000     kernel32:KERNEL32.dll
 0000:ffff7000       .debug$S                   0000000180000000     kernel32:KERNEL32.dll
 0000:ffff7000       .debug$S                   0000000180000000     kernel32:KERNEL32.dll
 0000:ffff7000       .debug$S                   0000000180000000     kernel32:KERNEL32.dll
 0000:ffff7000       .debug$S                   0000000180000000     kernel32:KERNEL32.dll
 0000:ffff7000       .debug$S                   0000000180000000     kernel32:KERNEL32.dll
 0000:ffff7000       .debug$S                   0000000180000000     kernel32:KERNEL32.dll
 0000:ffff7000       .debug$S                   0000000180000000     kernel32:KERNEL32.dll
 0000:ffff7000       .debug$S                   0000000180000000     kernel32:KERNEL32.dll
 0000:ffff7000       .debug$S                   0000000180000000     kernel32:KERNEL32.dll
 0000:ffff7000       .debug$S                   0000000180000000     kernel32:KERNEL32.dll
 0000:ffff7000       .debug$S                   0000000180000000     kernel32:KERNEL32.dll
 0000:ffff7000       .debug$S                   0000000180000000     kernel32:KERNEL32.dll
 0000:ffff7000       .debug$S                   0000000180000000     kernel32:KERNEL32.dll
 0000:ffff7000       .debug$S                   0000000180000000     psapi:PSAPI.DLL
 0000:ffff7000       .debug$S                   0000000180000000     psapi:PSAPI.DLL
 0000:ffff7000       .debug$S                   0000000180000000     psapi:PSAPI.DLL
 0000:ffff7000       .debug$S                   0000000180000000     java:java.dll
 0000:ffff7000       .debug$S                   0000000180000000     java:java.dll
 0000:ffff7000       .debug$S                   0000000180000000     java:java.dll
 0000:ffff7000       .debug$S                   0000000180000000     java:java.dll
 0000:ffff7000       .debug$S                   0000000180000000     java:java.dll
 0000:ffff7000       .debug$S                   0000000180000000     java:java.dll
 0000:ffff7000       .debug$S                   0000000180000000     java:java.dll
 0001:00000b84       doPrivilegedOpenProcess    0000000180001b84 f   VirtualMachineImpl.obj
 0001:00000d0c       jstring_to_cstring         0000000180001d0c f   VirtualMachineImpl.obj
 0001:00000f30       $$000000                   0000000180001f30     MSVCRT:amdsecgs.obj
 0001:00000f60       ?dllmain_crt_dispatch@@YAHQEAUHINSTANCE__@@KQEAX@Z 0000000180001f60 f   MSVCRT:dll_dllmain.obj
 0001:00000fb0       ?dllmain_crt_process_attach@@YAHQEAUHINSTANCE__@@QEAX@Z 0000000180001fb0 f   MSVCRT:dll_dllmain.obj
 0001:000010c8       ?dllmain_crt_process_detach@@YAH_N@Z 00000001800020c8 f   MSVCRT:dll_dllmain.obj
 0001:0000114c       ?dllmain_dispatch@@YAHQEAUHINSTANCE__@@KQEAX@Z 000000018000214c f   MSVCRT:dll_dllmain.obj
 0001:000013c8       capture_previous_context   00000001800023c8 f   MSVCRT:gs_report.obj
 0001:00001c70       $$000000                   0000000180002c70     MSVCRT:guard_dispatch.obj
 0001:00001c90       $$000000                   0000000180002c90     MSVCRT:guard_xfg_dispatch.obj
 0001:00001ca6       ?fin$0@?0??dllmain_crt_process_attach@@YAHQEAUHINSTANCE__@@QEAX@Z@4HA 0000000180002ca6 f   MSVCRT:dll_dllmain.obj
 0001:00001cbd       ?fin$0@?0??dllmain_crt_process_detach@@YAH_N@Z@4HA 0000000180002cbd f   MSVCRT:dll_dllmain.obj
 0001:00001cd6       ?fin$1@?0??dllmain_crt_process_detach@@YAH_N@Z@4HA 0000000180002cd6 f   MSVCRT:dll_dllmain.obj
 0001:00001cea       ?filt$0@?0??dllmain_dispatch@@YAHQEAUHINSTANCE__@@KQEAX@Z@4HA 0000000180002cea f   MSVCRT:dll_dllmain.obj
 0001:00001d20       __scrt_is_nonwritable_in_current_image$filt$0 0000000180002d20 f   MSVCRT:utility.obj
 0002:000005d0       GS_ExceptionPointers       00000001800035d0     MSVCRT:gs_report.obj
 0002:00000b40       $unwind$Java_sun_tools_attach_AttachProviderImpl_tempPath 0000000180003b40     AttachProviderImpl.obj
 0002:00000b60       $unwind$Java_sun_tools_attach_AttachProviderImpl_volumeFlags 0000000180003b60     AttachProviderImpl.obj
 0002:00000b74       $unwind$Java_sun_tools_attach_AttachProviderImpl_enumProcesses 0000000180003b74     AttachProviderImpl.obj
 0002:00000b88       $unwind$Java_sun_tools_attach_AttachProviderImpl_isLibraryLoadedByProcess 0000000180003b88     AttachProviderImpl.obj
 0002:00000bac       $unwind$sprintf            0000000180003bac     VirtualMachineImpl.obj
 0002:00000bb8       $unwind$Java_sun_tools_attach_VirtualMachineImpl_generateStub 0000000180003bb8     VirtualMachineImpl.obj
 0002:00000bcc       $unwind$Java_sun_tools_attach_VirtualMachineImpl_openProcess 0000000180003bcc     VirtualMachineImpl.obj
 0002:00000be8       $unwind$Java_sun_tools_attach_VirtualMachineImpl_createPipe 0000000180003be8     VirtualMachineImpl.obj
 0002:00000c04       $unwind$Java_sun_tools_attach_VirtualMachineImpl_connectPipe 0000000180003c04     VirtualMachineImpl.obj
 0002:00000c04       $unwind$__raise_securityfailure 0000000180003c04     MSVCRT:gs_report.obj
 0002:00000c04       $unwind$__scrt_initialize_crt 0000000180003c04     MSVCRT:utility.obj
 0002:00000c04       $unwind$__scrt_initialize_onexit_tables 0000000180003c04     MSVCRT:utility.obj
 0002:00000c04       $unwind$__scrt_release_startup_lock 0000000180003c04     MSVCRT:utility.obj
 0002:00000c04       $unwind$__scrt_uninitialize_crt 0000000180003c04     MSVCRT:utility.obj
 0002:00000c0c       $unwind$Java_sun_tools_attach_VirtualMachineImpl_readPipe 0000000180003c0c     VirtualMachineImpl.obj
 0002:00000c24       $unwind$Java_sun_tools_attach_VirtualMachineImpl_enqueue 0000000180003c24     VirtualMachineImpl.obj
 0002:00000c48       $unwind$doPrivilegedOpenProcess 0000000180003c48     VirtualMachineImpl.obj
 0002:00000c64       $unwind$jstring_to_cstring 0000000180003c64     VirtualMachineImpl.obj
 0002:00000c78       $unwind$jvm_attach_thread_func 0000000180003c78     VirtualMachineImpl.obj
 0002:00000c84       $unwind$__GSHandlerCheckCommon 0000000180003c84     MSVCRT:gshandler.obj
 0002:00000c8c       $unwind$__scrt_initialize_default_local_stdio_options 0000000180003c8c     MSVCRT:default_local_stdio_options.obj
 0002:00000c8c       $unwind$?dllmain_crt_dispatch@@YAHQEAUHINSTANCE__@@KQEAX@Z 0000000180003c8c     MSVCRT:dll_dllmain.obj
 0002:00000c8c       $unwind$DllMain            0000000180003c8c     MSVCRT:dll_dllmain_stub.obj
 0002:00000c8c       $unwind$__GSHandlerCheck   0000000180003c8c     MSVCRT:gshandler.obj
 0002:00000c8c       $unwind$__scrt_acquire_startup_lock 0000000180003c8c     MSVCRT:utility.obj
 0002:00000c8c       $unwind$__scrt_dllmain_after_initialize_c 0000000180003c8c     MSVCRT:utility.obj
 0002:00000c8c       $unwind$__scrt_dllmain_before_initialize_c 0000000180003c8c     MSVCRT:utility.obj
 0002:00000c8c       $unwind$__scrt_dllmain_crt_thread_attach 0000000180003c8c     MSVCRT:utility.obj
 0002:00000c8c       $unwind$__scrt_dllmain_crt_thread_detach 0000000180003c8c     MSVCRT:utility.obj
 0002:00000c8c       $unwind$__scrt_dllmain_uninitialize_c 0000000180003c8c     MSVCRT:utility.obj
 0002:00000c8c       $unwind$__scrt_dllmain_uninitialize_critical 0000000180003c8c     MSVCRT:utility.obj
 0002:00000c98       $xdatasym                  0000000180003c98     MSVCRT:amdsecgs.obj
 0002:00000c9c       $unwind$?dllmain_crt_process_attach@@YAHQEAUHINSTANCE__@@QEAX@Z 0000000180003c9c     MSVCRT:dll_dllmain.obj
 0002:00000cd8       $unwind$?fin$0@?0??dllmain_crt_process_attach@@YAHQEAUHINSTANCE__@@QEAX@Z@4HA 0000000180003cd8     MSVCRT:dll_dllmain.obj
 0002:00000cd8       $unwind$?fin$0@?0??dllmain_crt_process_detach@@YAH_N@Z@4HA 0000000180003cd8     MSVCRT:dll_dllmain.obj
 0002:00000cd8       $unwind$?fin$1@?0??dllmain_crt_process_detach@@YAH_N@Z@4HA 0000000180003cd8     MSVCRT:dll_dllmain.obj
 0002:00000ce0       $unwind$?dllmain_crt_process_detach@@YAH_N@Z 0000000180003ce0     MSVCRT:dll_dllmain.obj
 0002:00000d34       $unwind$?dllmain_dispatch@@YAHQEAUHINSTANCE__@@KQEAX@Z 0000000180003d34     MSVCRT:dll_dllmain.obj
 0002:00000d5c       $unwind$?filt$0@?0??dllmain_dispatch@@YAHQEAUHINSTANCE__@@KQEAX@Z@4HA 0000000180003d5c     MSVCRT:dll_dllmain.obj
 0002:00000d64       $unwind$_DllMainCRTStartup 0000000180003d64     MSVCRT:dll_dllmain.obj
 0002:00000d74       $unwind$__report_gsfailure 0000000180003d74     MSVCRT:gs_report.obj
 0002:00000d7c       $unwind$capture_previous_context 0000000180003d7c     MSVCRT:gs_report.obj
 0002:00000d88       $unwind$__security_init_cookie 0000000180003d88     MSVCRT:gs_support.obj
 0002:00000d94       $unwind$__scrt_is_nonwritable_in_current_image 0000000180003d94     MSVCRT:utility.obj
 0002:00000db4       $unwind$__scrt_is_nonwritable_in_current_image$filt$0 0000000180003db4     MSVCRT:utility.obj
 0002:00000dbc       $unwind$__scrt_dllmain_exception_filter 0000000180003dbc     MSVCRT:utility.obj
 0002:00000dd0       $unwind$__scrt_fastfail    0000000180003dd0     MSVCRT:utility_desktop.obj
 0002:00000de0       $unwind$_RTC_Initialize    0000000180003de0     MSVCRT:initsect.obj
 0002:00000de0       $unwind$_RTC_Terminate     0000000180003de0     MSVCRT:initsect.obj
 0002:00000dec       $unwind$__isa_available_init 0000000180003dec     MSVCRT:cpu_disp.obj
 0002:00000e00       $xdatasym                  0000000180003e00     MSVCRT:guard_dispatch.obj
 0002:00000e08       $xdatasym                  0000000180003e08     MSVCRT:guard_xfg_dispatch.obj
 0002:00000e10       .edata                     0000000180003e10     attach.exp
 0002:00000e38       rgpv                       0000000180003e38     attach.exp
 0002:00000e6c       rgszName                   0000000180003e6c     attach.exp
 0002:00000ea0       rgwOrd                     0000000180003ea0     attach.exp
 0002:00000eba       szName                     0000000180003eba     attach.exp
 0002:00000ec5       $N00001                    0000000180003ec5     attach.exp
 0002:00000efc       $N00002                    0000000180003efc     attach.exp
 0002:00000f3e       $N00003                    0000000180003f3e     attach.exp
 0002:00000f70       $N00004                    0000000180003f70     attach.exp
 0002:00000fa5       $N00005                    0000000180003fa5     attach.exp
 0002:00000fd8       $N00006                    0000000180003fd8     attach.exp
 0002:0000100e       $N00007                    000000018000400e     attach.exp
 0002:00001043       $N00008                    0000000180004043     attach.exp
 0002:00001077       $N00009                    0000000180004077     attach.exp
 0002:000010a8       $N00010                    00000001800040a8     attach.exp
 0002:000010de       $N00011                    00000001800040de     attach.exp
 0002:0000110c       $N00012                    000000018000410c     attach.exp
 0002:00001141       $N00013                    0000000180004141     attach.exp
 0002:00001570       .idata$6                   0000000180004570     java:java.dll
 0002:00001606       .idata$6                   0000000180004606     advapi32:ADVAPI32.dll
 0002:00001650       .idata$6                   0000000180004650     psapi:PSAPI.DLL
 0002:0000193a       .idata$6                   000000018000493a     kernel32:KERNEL32.dll
 0002:0000198a       .idata$6                   000000018000498a     vcruntime:VCRUNTIME140.dll
 0002:00001a8c       .idata$6                   0000000180004a8c     ucrt:api-ms-win-crt-string-l1-1-0.dll
 0002:00001aae       .idata$6                   0000000180004aae     ucrt:api-ms-win-crt-heap-l1-1-0.dll
 0002:00001ace       .idata$6                   0000000180004ace     ucrt:api-ms-win-crt-stdio-l1-1-0.dll
 0002:00001aee       .idata$6                   0000000180004aee     ucrt:api-ms-win-crt-runtime-l1-1-0.dll
 0003:00000040       _GetModuleHandle           0000000180005040     VirtualMachineImpl.obj
 0003:00000048       _GetProcAddress            0000000180005048     VirtualMachineImpl.obj
 0003:00000050       _IsWow64Process            0000000180005050     VirtualMachineImpl.obj
 0003:00000058       ?__proc_attached@@3HA      0000000180005058     MSVCRT:dll_dllmain.obj
 0003:00000060       GS_ExceptionRecord         0000000180005060     MSVCRT:gs_report.obj
 0003:00000100       GS_ContextRecord           0000000180005100     MSVCRT:gs_report.obj
 0003:000005f8       ?is_initialized_as_dll@@3_NA 00000001800055f8     MSVCRT:utility.obj
 0003:000005f9       ?module_local_atexit_table_initialized@@3_NA 00000001800055f9     MSVCRT:utility.obj
 0003:00000600       ?module_local_atexit_table@@3U_onexit_table_t@@A 0000000180005600     MSVCRT:utility.obj
 0003:00000618       ?module_local_at_quick_exit_table@@3U_onexit_table_t@@A 0000000180005618     MSVCRT:utility.obj
 0005:00000060       $R000000                   0000000180007060     attach.dll.res
